:020000040000FA
:10000000831619309900243098008312903098009C
:1000100083168610831286144320A00050302002DD
:1000200003191F2849302002031922284C302002CE
:1000300003192B2853302002031933280C284F3082
:1000400047200C28493047202030472030304720B7
:10005000003047200C2839200008A3004C304720EE
:10006000230847200C2839204320800053304720A4
:100070000C28432084004320A10021184128831329
:100080004228831708008C1E43281A0808000C1EFB
:060090004728990008005A
:00000001FF
